:020000040000FA
:0600000000308600072815
:08000800AD0A0B1109000313FE
:10001000831207309F00A0308B00103085008316BC
:1000200000308600C5308100043085008312203006
:1000300084008001840A041F19280030AB001922B3
:100040002130D523AE002430D523B1002230D52372
:10005000B800B3000230D523BE001E30D523C00047
:100060002330D523AC00AC182C150430B5003C125D
:100070000510E9212930C2002E08C100BF23C62087
:100080009120FF2027223F28043005052A06031966
:10009000B90A08002A1D4F28051D4C28080005191B
:1000A0004F2808002A194F284C28AD01752004302C
:1000B00005052A0603195F28AD186E2856287520F5
:1000C00075207520B90144207520752044207520C5
:1000D000E120442085110230390208002030C2009E
:1000E0002F08C100BF234A2020282B1884288611FE
:1000F000010C7F39031980282F02031C0611080008
:10010000AF08031D061508000611010C7F390319FD
:100110008D282F02031C86110800AF08031D8615C9
:1001200008002508A1002608A2002708A300280827
:10013000A400A501A601A701A80125308400A320E1
:10014000AB20B32008000830A90052205520800DB4
:10015000A90BA5280800840A52205520800D5220A2
:100160005520800D0800840A0430A9005220552033
:10017000800C840A52205520800CA9030319C22840
:100180008403B628800E8403800E08002030B90056
:100190001330A900043005052A060319D428B90B29
:1001A000D7280430AA06C6282A30A900CF28043050
:1001B00005052A060319C8287520E120A90BD728B0
:1001C0000800BC1CFC2832082F02031CFA2803106C
:1001D0003B0D2C1C3B08323E2C180A3EA000010CA3
:1001E000A002031808007D3C031CF8280510080035
:1001F0000514080005147528AC1805107528851518
:1002000021082502031D202922082602031D20297A
:1002100023082702031D202924082802031D202962
:1002200021082E0203191A292C1F20292108310226
:10023000031D20297520230824020319AD29212933
:1002400008003C162808FE3E03194829FF3E031902
:100250000613FF3E03198613FF3E03194E29FF3E86
:1002600003199921FF3E03197E21FD3E03195329ED
:10027000FF3E03190617FF3E03198617FF3E0319B9
:100280004B29FF3E0319A321FF3E03198C21C729E7
:100290002308073C72292308F83E72292308073CEB
:1002A00003186629722908302702031C72290319D2
:1002B0002029FD3E03190617FF3E03198617FE3E4F
:1002C0000319A321FF3E03198C21C72903197E219D
:1002D000FF3E03199921FE3E03198613FF3E0319C1
:1002E0000613C729240801392B060319C729240836
:1002F0000139AB0021220130A300C729AC1E8A2995
:10030000BC1E0800B9002230D523B800B300BC12CF
:100310003908080085100800AC1E9729BC1A08008F
:10032000B9000130B800B300BC16390808008514C4
:1003300008002C1DA129AC1C9F29BC1008003C11F1
:100340000800051008002C1DAB29AC1CA929BC1401
:1003500008003C1508000514080075202308013A20
:10036000031DC2293C18B829FF30B4000430B50081
:100370003C186B223C18C7293C14AB090130AB0573
:100380002122C729AC18BC143C1CC7293C1075207D
:10039000E9212308013A0319E6292308BB003C1987
:1003A000DE290310BB0DAC1FE229A2080319E229C4
:1003B000221CBB0AA218E229BB0AE2293C1EE22940
:1003C0003030BB073B08D523B2000800B201AF01B3
:1003D00008002C1A0B2A2B18FC2906128616AF08C7
:1003E00003198612AC1D86163C1A0800A218FA29B9
:1003F000061308000617080086120616AF08031930
:100400000612AC1D06163C1A0800A218092A86130B
:100410000800861708002B18132A0612A218861641
:10042000A21C861208008612A2180616A21C06122A
:1004300008002030D523AF00B2002530D523AB0013
:1004400008002530C2002B08C100BF23080038086F
:10045000013C031D2E2A3208AF0008003C1232086E
:100460002F0203190800B30B08003E082F020318DF
:10047000422AB20803193F2A3E08AF00422AAF01C0
:10048000B30A080032082F02031C482AAF03492A86
:10049000AF0A3808B300AD012630D5232F08BF00BE
:1004A000C10B532A572ABF070318AD0A502A04303C
:1004B000C100AD0CBF0CAD13C10B592AAD08031818
:1004C000632AAD0CBF0C2730D5233F084102031C23
:1004D0000030B3070800B40B08006F2A0800FF3093
:1004E000B400B50B0800A52AB600B60A0B30BC1B39
:1004F000DB2BB60B7C2A080086160616DB23861239
:100500000612DB23792A0230B6002F30772A922296
:100510002308013A0319872A92222308013A031D6E
:100520008C2A0800C620912021082502031D922A4A
:1005300022082602031D922A23082702031D922A5D
:1005400024082802031D922A0800BC1009307422D6
:10055000013074228722E123B9030319D62AB90393
:100560000319DE2AB9030319E92AB9030319232B56
:10057000B9030319392BB9030319912BB9030319D3
:10058000992BB90303196C2BB90303197F2BB903FA
:1005900003194B2BB90303195E2B0430B90203195D
:1005A000AB2B21080319B72B8322AA2A7422872296
:1005B0002130C2002108C100BF23A82A742287224B
:1005C0002230C200E1233908C1002230C200BF231B
:1005D000A82A74228722E123C2000310C20D210839
:1005E0000319082B10303902031CF82A8322EA2A47
:1005F000390874228722E1230310B90DB91F022B99
:100600008322FA2A3908C100BF2301307422EA2A62
:100610000630B600D523B900B6033603D523B90298
:100620000310390CC1073608C200BF2383169C187B
:10063000172B8312B60A1E3036020318A82AB60AF0
:10064000B60A36080A2B74228722E12304303902C5
:10065000031C2C2B8322242B2330D523E730C10508
:10066000B9033918C115B91841162330C200BF2388
:10067000A82A74228722E12303303902031C422B6B
:1006800083223A2B2330D523C112391CC1162330C3
:10069000C200BF23A82A74228722E1230430390232
:1006A000031C562B21303902031C582B83224C2B60
:1006B0002630C2003908C100BF23A82A742287222D
:1006C000E123B908031D662B83225F2B2730C2006C
:1006D0003908C100BF23A82A74228722E1230530EC
:1006E0003902031C752B83226D2B2330D523F83060
:1006F000C1053908C1042330C200BF23A82A7422CF
:100700008722E12303303902031C882B8322802BAC
:100710002330D523C113391CC1172330C200BF2396
:10072000A82A742287222430C2002108C100BF23D6
:10073000A82A74228722E12303303902031CA22B4A
:1007400083229A2B2330D5234113391C41172330A0
:10075000C200BF23A82A8722E12303303902031CE9
:10076000B32B8322AB2BBC13391CBC17A82AFF3038
:10077000B4000430B50001307422912120284108D2
:1007800083169A008312420883169B008B131C1257
:100790009C111C1555309D00AA309D009C141C1105
:1007A0009C18D02B83128B17080083169B001C14F7
:1007B0001A0883120800AD01AD02AD08031DDD2B40
:1007C0000800B901A11FE72BB90A211FB90AA11E10
:1007D000ED2B0330B907211EB907A11DF32B0930FA
:1007E000B907211DB907A11CF92B1B30B907211C22
:0607F000B90739080800FA
:02400E00703F01
:104200000000000012000000140015001600180045
:104210001A001C001E0020002200250028002B0090
:104220002E00320036003A003E00430048004E00A7
:1042300054005A00600067006E0075007C000000AA
:1042400000002A0003002000A900000010001E004A
:10425000000000000000000000000000000000005E
:104260000000000008000A000C000E001000120000
:10427000150018001B001E002100250029002D003C
:00000001FF
